:1000000012C0189518951895189518951895189563
:100010001895189518951895189518951895189578
:100020001895189518958FED8DBFC0ECE0EC4E2E0D
:10003000DD275D2EEEE7F0E0A0E6B0E0A89584B7FE
:10004000082E877F84BF88E1992781BD91BD8827CD
:100050008D933197E9F7D5D266248FE087BB8FEF78
:1000600081BB80E082BB8FE788BB8CE012D3BF9856
:10007000A6E69C9197FF04C0B7990EC09F779C930A
:10008000B79B0AC088E29F9399272FD39F91B79B74
:1000900003C090689C9347D29AD2E0E6F7E08FD2F3
:1000A000E2E0F0E0A5D291D2E0E7F7E088D2E2E02A
:1000B000F0E09ED280E080936400A1E629D380E046
:1000C0008093630080E08093650081D2E0E8F7E0F0
:1000D00076D2C09AC39881E080936000BE98A6E66D
:1000E0009C9196FF04C0B69B0EC09F7B9C93B699D3
:1000F0000AC088E29F939927F8D29F91B69903C0CE
:1001000090649C9313D182E080936000BD98A6E632
:100110009C9195FF04C0B59B0EC09F7D9C93B599A3
:100120000AC088E29F939927E0D29F91B59903C0B6
:1001300090629C93FBD083E080936000BC98A6E61D
:100140009C9194FF04C0B49B0EC09F7E9C93B49975
:100150000AC088E29F939927C8D29F91B49903C09F
:1001600090619C93E3D0C39AC29884E0809360002E
:10017000BE98A6E69C9196FF04C0B69B0EC09F7BDE
:100180009C93B6990AC088E29F939927AED29F911B
:10019000B69903C090649C93C9D085E080936000B9
:1001A000BD98A6E69C9195FF04C0B59B0EC09F7DAF
:1001B0009C93B5990AC088E29F93992796D29F9104
:1001C000B59903C090629C93B1D086E080936000A3
:1001D000BC98A6E69C9194FF04C0B49B0EC09F7E81
:1001E0009C93B4990AC088E29F9399277ED29F91ED
:1001F000B49903C090619C9399D0C29AC19887E04A
:1002000080936000BE98A6E69C9196FF04C0B69BC2
:100210000EC09F7B9C93B6990AC088E29F93992752
:1002200064D29F91B69903C090649C937FD088E07C
:1002300080936000BD98A6E69C9195FF04C0B59B95
:100240000EC09F7D9C93B5990AC088E29F93992721
:100250004CD29F91B59903C090629C9367D089E07E
:1002600080936000BC98A6E69C9194FF04C0B49B68
:100270000EC09F7E9C93B4990AC088E29F939927F1
:1002800034D29F91B49903C090619C934FD0C19A8E
:10029000C0988BE080936000BE98A6E69C9196FF84
:1002A00004C0B69B0EC09F7B9C93B6990AC088E29F
:1002B0009F9399271AD29F91B69903C090649C93FB
:1002C00035D08AE080936000BD98A6E69C9195FFAA
:1002D00004C0B59B0EC09F7D9C93B5990AC088E26F
:1002E0009F93992702D29F91B59903C090629C93E6
:1002F0001DD08CE080936000BC98A6E69C9194FF92
:1003000004C0B49B0EC09F7E9C93B4990AC088E23F
:100310009F939927EAD19F91B49903C090619C93D0
:1003200005D08AE090E0E1D1D4CE9FCE939A84E6C6
:1003300090E0DBD1939882E390E0D7D10091640004
:10034000013009F001C048C000916400023009F09A
:1003500001C067C0009160000B3009F02AC0A6E31D
:100360000C9104FB81E00EF480E08F93A6E30C91E6
:1003700005FB81E00EF480E09F91892B8F93A6E32B
:100380000C9106FB81E00EF480E09F91892B88237D
:1003900009F401C0E4CF1BD1E0E9F7E010D1A4E6F5
:1003A0008C918F5F8C9380E0809363008FE788BB94
:1003B00090CE009160000C3009F00DC0EAE0F0E052
:1003C000A4E1C6D1A1E60D911C910417150709F00F
:1003D00001C091C069C03AC0009160000C3009F0C2
:1003E0001FC0EAE0F0E0A4E1B3D1A1E60D911C91B9
:1003F0000417150709F401C057C0A1E689D180E0B0
:100400008093630080E080936500A4E68C918F5F09
:100410008C93DDD0E0EAF7E0D2D08FE788BB59CEED
:1004200015C0009160000C3009F010C0EAE0F0E067
:10043000A1E67BE77CD1CBD0E0EBF7E0C0D04AD09F
:10044000E2E0F0E0D5D08FE788BB34CEA3E68C9114
:100450008F5F8C930091630046E0040FA5E60C9338
:100460008FEBA5E61C91C2D0E0ECF7E0A8D000919C
:100470006300043010F009F001C001C015C0A1E60E
:100480000D911C914AE050E087D0A1E60D931C939A
:10049000A1E60D911C91A0E64D915527040F151F63
:1004A000A1E60D931C93089592D0E2ECF7E087D07B
:1004B00084E690E01AD18FE788BB939AE3E0F0E0FE
:1004C00097D0939882D0E0E6F7E079D0E4E1F0E0CD
:1004D0008FD0F0CD84E690E008D1939A88EC90E03C
:1004E00004D1939888EC90E000D1939A88EC90E046
:1004F000FCD0939808956BD0E0EBF7E060D0EADF92
:1005000064D0E0EDF7E05BD08CE291E0EED08FE7D5
:1005100088BB949AE1E0F0E06BD0949858D0E1E089
:10052000F0E066D0C7CDB79901C014C0EAE0F0E0B2
:1005300002ED14E0A0E1BB277BE7F9D0CBDF47D089
:10054000EEEDF7E03CD041D0EEEEF7E038D0E5E05C
:10055000F0E04ED0AFCD04D01FD000FC0CD00895F9
:100560000024E89457FF02C009D0689400F80BD02B
:1005700010F80124089502D009D0089550954095AF
:100580004F5F5F4F0895E89417FF08950095109509
:100590000F5F1F4F68940895752F642F55274427C8
:1005A000FF93F1E1889405C010F4460F571F56954C
:1005B000479517950795FA95B9F7FF910895A4D037
:1005C000802D11F060D0FBCF089580EC62C081E0F7
:1005D00060D014D080E85DC08FE7213039F08FEB18
:1005E000223021F08FE8233009F08FEC810F51C0C9
:1005F00088EE93E07AD03197D9F7089583E0992770
:1006000074C08AEF90E071D0BB9ABA9AB99AB89A3E
:100610008E9A8D9A959885E090E067D09698C398C9
:10062000C298C19AC09A969AEF93FF93E5E1F0E0E1
:1006300050D0FF91EF91969855D0969AEF93FF93F3
:10064000E5E1F0E046D0FF91EF9196984BD0969A75
:10065000EF93FF93E5E1F0E03CD0FF91EF919698A6
:1006600041D0C098969AEF93FF93E5E1F0E031D046
:10067000FF91EF91969836D088E20BD08EE009D0AA
:1006800086E007D00895959A829505D004D02AD0A7
:1006900008959598F9CF859510F4C09A01C0C09837
:1006A000859510F4C19A01C0C198859510F4C29A3D
:1006B00001C0C298859510F4C39A01C0C398969A58
:1006C000EF93FF93E5E1F0E004D0FF91EF9196986E
:1006D00008953197F1F70895689462F80895E894C1
:1006E00062F8089581E090E000C0EF93FF93EE2759
:1006F000E82BE92B31F0EAEFF0E03197F1F70197C1
:10070000D1F7FF91EF910895C89531960020089593
:1007100082E001C084E099279D938A95E9F70895C6
:10072000E199FECFEEBB3196089591E001C092E0D1
:100730007B3751F47FB7F894F3DF8D918DBBE29A4C
:10074000E19A9A95C9F77FBF7727089591E001C094
:1007500092E0E6DFE09A8DB38D939A95D1F70895F4
:100760005757572E4156522E344D472E434F4D006A
:100770002020436F64654C6F636B4156522020000C
:10078000202020456E74657220636F646520000030
:1007900020456E746572206F6C6420636F64650021
:1007A00020456E746572206E657720636F64650006
:1007B00020436F6465206163636570746564000045
:1007C0002A00202020436F64652077726F6E6700D7
:1007D00020202020556E6C6F636B65640000202024
:1007E000496E697469616C20636F64650000202044
:0E07F000202020697320202031323334000095
:00000001FF
